:100000000EC01DC01CC01BC021C019C018C017C025
:1000100016C015C014C013C012C011C010C01124E6
:100020001FBECFE5D2E0DEBFCDBF10E0A0E6B0E05E
:1000300001C01D92A936B107E1F704D064C0E0CF3A
:10004000089508954CD0FCDFFCDFFECF1F920F9285
:100050000FB60F9211242F933F938F939F93AF93DB
:10006000BF938091640090916500A0916600B0916B
:10007000670030916800232F2D5F2D3728F02D5712
:100080000296A11DB11D03C00196A11DB11D2093B3
:1000900068008093640090936500A0936600B0931D
:1000A00067008091600090916100A0916200B09122
:1000B00063000196A11DB11D8093600090936100C3
:1000C000A0936200B0936300BF91AF919F918F9115
:1000D0003F912F910F900FBE0F901F90189578941D
:1000E00080B7806880BF80B7806480BF8CB5806433
:1000F0008CBD8FEF8DBD80B7807F876080BF89B753
:0A010000846089BF0895F894FFCFD2
:00000001FF
